:020000040000FA
:10000000702AFF3FFF3FFF3F0800831203132E08B3
:10001000B4003106B5002F08031D32080319582813
:1000200083120313AF077E30031C1A28AF02031C90
:100030001F285C2883120313AF02031C5528831268
:1000400003132D08B300B417B117AD01AE01103082
:10005000B60083120313B40CB30C031C352830080C
:10006000AD0731080318310FAE0783120313AE0C2E
:10007000AD0CB60B2928AE1B4628AD0DAE0DAF0852
:100080000319552883120313AF03340D831203138E
:10009000371F6628031C6628AD0F6628AE0F66283A
:1000A000AE0CAD0CAF0F66285C2883120313371516
:1000B00083120313AF01612883120313B714FF30B7
:1000C000AF0083120313AD018030AE00831203131F
:1000D000B51FAE13831203132D08080083120313F8
:1000E00032082F02B50003188928B509B50A2F0870
:1000F000B4003208AF003408B2002E08B400310852
:10010000AE003408B1002D08B4003008AD0034084A
:10011000B0001230831203133502031833298312FF
:100120000313B2080319332983120313B3012E08F2
:10013000B4002E083106B600AE17B117083083128E
:100140000313B502031CAC28831203133008B30059
:100150003108B000B1019E2883120313B5070319BB
:10016000B928031083120313B10CB00CB30CB50BF8
:10017000B12883120313B61F00293008AD023108DD
:10018000031C310FAE020318CC28AE09AD09AD0A2D
:100190000319AE0A8030B40683120313B309B30AFD
:1001A0000319D628AD032D0A0319AE0303308312B9
:1001B0000313B50083120313AE08031DED282D08A9
:1001C000AE003308AD00B3010830AF02031C212993
:1001D00083120313B50BDA28212983120313AE1BF4
:1001E000F8280310B30DAD0DAE0DAF0BED2821298E
:1001F00083120313371F2F29B31F2F29B301182987
:10020000831203133008AD0731080318310FAE070E
:10021000031C122983120313AE0CAD0CB30CAF0AEE
:100220000319252983120313371F2F29B31F2F29E1
:1002300083120313AD0F2F29AE0F2F2903142D1096
:100240000A2983120313AF012A2983120313B71457
:10025000FF30AF0083120313AD018030AE00831274
:100260000313B41FAE13831203132D0808008E303E
:1002700083120313B300B401B501AF1F4A29AF09BC
:10028000AE09AD09AD0F4729AE0A0319AF0A8312B3
:100290000313B51783120313AF0803195829083045
:1002A000B3072D08B4002E08AD002F08AE006D294D
:1002B00083120313AE08031D6D290830B3022D0805
:1002C0000319832983120313AE00AD016D29831234
:1002D0000313B40DAD0DAE0DB30383120313AE1FA4
:1002E0006729371F7D29B41F7D29AD0F7D29AE0FEA
:1002F0007D290314AE0CAD0CB30A8312031333082B
:10030000AF00B51FAE13831203132D08080083122C
:1003100003132E08B3007E302F02B400031CC9293A
:1003200083120313AE17AF01B5013408103CB400BB
:100330000318A6290830B407031CC4298312031329
:100340002E08AF002D08AE00AD01B229083083128F
:1003500003133402031CB229B4002D08B5002E0883
:10036000AD00AE0183120313B4080319C0290310B2
:1003700083120313AF0CAE0CAD0CB50CB40BB72944
:1003800083120313AF1FD12983120313B714FF3055
:10039000CA29000183120313AD00AE00AF00AF13F2
:1003A000E62983120313371FDA29B51FDA29AD0AAC
:1003B0000319AE0A83120313B31FE629AF09AE096E
:1003C000AD09AD0FE629AE0A0319AF0A8312031374
:1003D0002D08080003108312031332082F04031999
:1003E000080083120313AE1B042AB11B142A8312C4
:1003F00003132D0830022E08031C2E0F31022F0884
:10040000031C2F0F3202142A83120313B11F08009A
:100410008312031330082D023108031C310F2E0202
:100420003208031C320F2F02031C182A0310080085
:100430000314080083120313AA01AB01AC01831259
:1004400003132A08AD002B08AE002C08AF00B00142
:10045000B1017F30B2006E20831203132D08AA0071
:100460002E08AB002F08AC002A08AD002B08AE0008
:100470002C08AF002708B0002808B1002908B200F6
:10048000EA21031C1F2A080083120313A701A801F5
:10049000A9019F149F184A2A831203131E08AD0056
:1004A000AE01AF013721831203132D08A7002E08D8
:1004B000A8002F08A900270808008312031385014C
:1004C000FF308316850070309F00013083120317C0
:1004D0009E00013003139F008701831687010800E7
:1004E0005D2283120313A001A1017F30A200A301AA
:1004F000A401A501A6012008AD002108AE00220834
:10050000AF008721831203132D0887004422831232
:1005100003132708A4002808A5002908A60024081A
:10052000AD002508AE002608AF00B0014030B10094
:100530008230B2000520831203132D08A4002E0878
:10054000A5002F08A600A308031DCE2A2408A70093
:100550002508A8002608A9001A2283120313A20F57
:10056000B32AB714A20383120313A11BC12A2008C4
:100570002104031DC12A2208823A031DC12A013029
:10058000A300831203132008AD002108AE00220847
:10059000AF008721831203132D08870083120313F2
:1005A000230B862A2408A7002508A8002608A900EE
:1005B0001A2283120313A20803193715031DA2037D
:1005C000A11BEA2A20082104031DEA2A22087F3AF7
:1005D0000319A301831203132008AD002108AE0004
:1005E0002208AF008721831203132D088700862A73
:1005F000FF3FFF3FFF3FFF3FFF3FFF3FFF3FFF3F0B
:10060000FF3FFF3FFF3FFF3FFF3FFF3FFF3FFF3FFA
:10061000FF3FFF3FFF3FFF3FFF3FFF3FFF3FFF3FEA
:10062000FF3FFF3FFF3FFF3FFF3FFF3FFF3FFF3FDA
:02400E00D430AC
:08400000FF3FFF3FFF3FFF3FC0
:00000001FF
